:020000020000FC
:0200000003C03B
:1000060088C00FEF01BB00E002BB00E004BB0CE3BD
:1000160005BB0FE307BB0CEF08BB0FE50DBF04E004
:100026000EBF41E051E071E088279927AA27BB2738
:10003600CC27DD2709E005BD09EF03BD00E809BFB0
:1000460000E905BF00E808B903E806B97894889581
:10005600FECF00E002BB0CEF08BB0CE305BB871725
:1000660008F0C298072F065F801708F0C398971705
:1000760008F0C498072F065F901708F0C59803B3D9
:1000860002FD10C0A71709F4C298072F065FA01734
:1000960009F4C398B71709F4C498072F065FB01779
:1000A60009F4C598072F0A95EDE5F0E0E00F002763
:1000B600F01F099409C00AC00BC00CC00DC00EC0C9
:1000C6000FC010C011C012C0909A0895919A089559
:1000D600929A0895939A0895949A0895959A0895F0
:1000E600969A0895979A0895C09A0895C19A089580
:1000F600803009F08A95903009F09A95C03011F059
:10010600CA9501C0A82FD03011F0DA9501C0B92FD9
:10011600089524B135B1062F0170006C07B9369ADF
:10012600002710E02B30310778F1039510E02E30D0
:10013600310750F1039510E02231310728F103957C
:1001460010E02631310700F1039510E02C3131071C
:10015600D8F0039510E024323107B0F0039510E093
:100166002D32310788F0039510E02833310760F00F
:10017600039510E02734310738F0039510E02A354F
:10018600310710F0039501C032C010E02137310766
:1001960070F1039510E02E38310748F1039510E011
:1001A600233B310720F1039510E0213E3107F8F09B
:1001B600039511E02B313107D0F0039511E0243679
:1001C6003107A8F0039511E0213C310780F0039533
:1001D60012E02533310758F0039512E0273C31072A
:1001E60030F0039513E02F37310708F00395639538
:1001F60060FD08C0801708F4802F0A1710F0C3E4CA
:10020600A02F07C0901708F4902F0B1710F0D3E417
:10021600B02F4A9549F440E21CDF7A9529F47AE03A
:0A0226005A9511F453E064DF1895B7
:00000001FF
